:020000040000FA
:0200000038289E
:08000800A000030E8312A10009
:10001000063081070B11C803C00B0F28C103A20BC8
:100020002028C830A2003A08031DBA03A30B2028D9
:100030000A30A3003F08031DBF033B08031DBB0399
:10004000210E8300A00E200E09002034203420341D
:100050007334733477342E34613473346D34203414
:10006000563431342E343634203420342034203485
:100070008316FF23900083128501831632309F0080
:1000800080308100FB30DF39FE398500831220305B
:1000900084008001840A841F4928A20AA30AFF3031
:1000A00081008B168B1748212608C3002708C4003F
:1000B000391539088500CC20051A602857223714D5
:1000C000391185018316A8309900831203309900F5
:1000D00037189F2A2408A504031DC62B3230B920E7
:1000E000031CB7143430B920031C37151E212F0808
:1000F0000319B715BB00B71A8228B71982283B0825
:1001000003198728CD20381A8A2837127B28851DA5
:1001100037178D28371A7B28B711B91608222C08F3
:1001200003199528BA002830AE202D0803199B2802
:10013000BA002A30AE20B91208222E08BA002630A2
:10014000AE203716B71EA628B712A828851DB716E9
:10015000371F77283713381E8D287728840000082A
:10016000C300840A0008C400CD203A08031DB42847
:10017000080084003008800731080318013E840A13
:1001800080070310800C8403800C300800023108C3
:10019000031C013E840A00020800E421B810381153
:1001A0001E213818ED2832080E023308031C013EC8
:1001B0000F02B71CDE28031CB814E0280318B8147B
:1001C00034080E023508031C013E0F02371DEB28D0
:1001D000031C3815ED28031838153808BC06BC1C5C
:1001E000F4280530BE00FC283E080319FC28BE0B8D
:1001F000FC283812B81838163C1D01293608BF00F3
:100200000A29360803190A293F08031D0A29B812CA
:100210003819B8163C1C0F291430BD0017293D08A9
:1002200003191729BD0B1729B8113818B815380844
:10023000BC00B819B715B81AB71508003810C001B6
:100240000030C1003330C0008E018F01413090007A
:100250004421381808000E080F04031928294421E6
:100260003818080009300F0203183E29051E2F29EF
:10027000900103300F02031C242908004421381880
:100280000800051E3E2924296400C11B38140800FB
:100290002630840000309721031D24142830840068
:1002A00003309721031DA4142A30840006309721BF
:1002B000031D24152C30840009308B21031DA41547
:1002C0002D3084000B308B21031D24162E3084002A
:1002D0000D308B21031DA4162F3084000F308B218D
:1002E000031D24173030840011309721031DA417FB
:1002F0003230840014309721031D251434308400DB
:1003000017309721031DA514363084001A308B2135
:10031000031D25150800C200AC218000420AAC2153
:100320000006FF3A03190800800103110800C2000B
:10033000AC218000840AC20A4208AC218000420A33
:10034000AC2100068403000603190800DC3080009D
:10035000840A05308000080083169B001C141A08CC
:1003600083120800C200CA210008CF21C20A840AF1
:100370004208CA210008CF21420ACA21000884038A
:100380000006CF29C200CA210008CF21420ACA2193
:100390000009CF2983161C159B00831208008B13BC
:1003A00083169A0055309D00AA309D009C1483123C
:1003B00064008C1FD8298C1383161A081C111C1476
:1003C0001A0683128B1708008B13900143098E00C5
:1003D00044098F00390801388500013090008B17DF
:1003E0000F0FF0298E1FF2298B130E080339031902
:1003F000012AFF3E0319012AFF3E0319012A002AA0
:10040000012A00008F1B012A390885008B179001F3
:1004100008005F300E020530031C013E0F02031C72
:10042000451559300E020630031C013E0F02031819
:10043000C515080045084A060C39031D2E2A4B082D
:1004400003190800CB0B080045192A2AC5192C2AC4
:10045000C51608004516080045170800CA060530ED
:10046000CB008F30C5050800051E3D2A392A851DA1
:100470003D2AC70B0800C51408000A30C700C51084
:100480000800E4216400C81F422A2730C800C90BB5
:100490000800451408004511C511E4211E21381C2F
:1004A00009221A22C81F08002830C807472A0A3024
:1004B000C700C510B91A612A0530C900B916451020
:1004C000652A0530C900B91245103422C5186C2AB6
:1004D0004122451C652A5A2AB912390885000800AC
:1004E0000A30C700C510B91A7A2A0530C900B916F2
:1004F00045107E2A0530C900B91245103722C518AB
:10050000852A4122451C7E2A732AB91239088500A2
:100510001E210800B91A912A0530C900B9164510E4
:10052000952A0530C900B91245104B22C51A9B2ADD
:10053000451C952A8A2AB91239088500080001301D
:10054000CC000530CB0070228A224C3084000B3066
:10055000F622702255234618EE2AC618B22A4619EA
:10056000DE2AA52A0030C900B91645100008C300CC
:10057000840A0008C4004B22851DD42A4519CA2AC2
:10058000C519C32ABB2AC30FC62AC40A4408083C9B
:100590000318BB2A0130C3020318013CC4024408FB
:1005A000023C031CBB2AC32A44088000840343087E
:1005B00080002608C3002708C400F02A0030C900C4
:1005C000B91645104B22851DE62AE22A3818F02A72
:1005D0000E088000840A0F088000F02A6330F6229B
:1005E000B9123908850082237022A52ACE00D101D4
:1005F000CF01D00100080319072BCD00D00A500805
:100600000A3A031D052BCF0AD001CD0BFE2A511843
:10061000112B51143230C900B91245100130CD00F0
:100620002F2BD1181E2BD1144F080319262BCD00C8
:10063000CD070A30C900B91645102F2B5119262BAA
:1006400051151E30C900B91245100E2BD1015008AA
:10065000031D172B1E30C900B91645100E2B4B2257
:10066000851D0800451A472B451B4E2B451C2F2B7B
:10067000CD030319072BB91A422B0A30C900B9164A
:1006800045102F2B0A30C900B91245102F2B8003BB
:100690000009031D532B4E088000532B800A0008CD
:1006A0004E02031C80018A22F72AC60103308A0009
:1006B0004C088207CC28662B6A2B6C2B6E2B722B76
:1006C000742B762B782B7C2B7E2B802B2630840072
:1006D000C61408002830672B2A30672B2C30840082
:1006E000461408002D306F2B2E306F2B2F306F2BC0
:1006F00030308400461508003230792B3430792BA5
:1007000036306F2B4C0382078F2B942B992B9E2B0B
:10071000A32BA82BAD2BB22BB72BBC2BC12B263078
:1007200084000030B2210800283084000330B22158
:1007300008002A3084000630B22108002C308400E2
:100740000930C22108002D3084000B30C22108007E
:100750002E3084000D30C22108002F3084000F306D
:10076000C2210800303084001130B221080032303C
:1007700084001430B2210800343084001730B221D4
:100780000800363084001A30C22108000130E4230A
:100790000230E4230430E4230830E4231030E4235F
:1007A0002030E4234030E4238030E4230130E6238A
:1007B0000230E6230430E6233C30C900B91245106C
:1007C0004122451CE02BC62B2405E72B2505031DE4
:1007D000EE2B0A30C900B9164510F22B1E30C900A5
:1007E000B91645104122451CF22B0A30C900B91236
:0A07F00045104122451CF92B0800BA
:02400E00CC3FA5
:10420000DC000500D900DC000500D900D60006005E
:10421000D0000000FF000500FA000A00F50037009A
:10422000C800DC000500D900080007000F00B0003E
:084230000400B4000A00F500CF
:00000001FF
